:10000000000005308A00522DFF0003088301FE0026
:100010000408FC000A08FD0015308A00CE2D831369
:10002000C000C101C10D003041027C300319400203
:10003000031C2028BD1B20282430C0070318C10A38
:1000400000304102F03003194002031C2C288317B2
:100050002030C0070318C10A013041027030031973
:100060004002031C35282030C007400884000800E7
:100070008030A100FE305A2101305A217530B10084
:100080003030BD29A101A117BF00FE305A213F0821
:100090005A29A601B800B901A01126080319A01514
:1000A0000530A5002730B500103062200330B500C0
:1000B000E8306220B50164306220B5010A30622068
:1000C00038086928B4003908B1003808B000462261
:1000D0003008B000A5030319A011260803197328DE
:1000E000250203187A283008031DA011A0197A28C8
:1000F000303E5A290800CD00C31F80282D305A21D8
:10010000A801A901AA01AB01C3176A30C2070310F5
:10011000C30CC40CC50CAB0CAA0CA90CA80CC20FC8
:10012000872845084202C507C20244084302C407A3
:10013000C302A601D3202E305A21CE010310280D70
:10014000C500290DC4002A0DC3002B0DC200CE0D21
:100150000310C50DC40DC30DC20DCE0D2808C50773
:1001600029080318290FC4072A0803182A0FC307F0
:100170002B0803182B0FC2070318CE0F0310C50D51
:10018000C40DC30DC20DCE0D4E08303E5A21450898
:10019000A8004408A9004308AA004208AB00CD0B00
:1001A0009D280310782AA0112608031DDA28A0151F
:1001B0000A30A6004508B3004408B2004308B10065
:1001C0004208B000A501BB01BA01B9010A30B8006C
:1001D000CC21A50A25082602031DE3283808031DA3
:1001E000A011A01DF528260BF8283808303E5A210A
:1001F000A60BDA28782AB80025080319782A3918B6
:10020000831738088400000883130319782A5A21B9
:10021000B80AA503FC28BD008611061183168611B5
:1002200006110F30860583123D08A01835293E308F
:10023000B1008030BD213330BC0049211330B10002
:100240008830BD2149216430BC2149216430BC2162
:100250002230BC004921283034210C3034210630B2
:100260003421A0143D0835292014BC00201C43294A
:100270000611033C031C482948210730B100D03047
:10028000BD21031408002014FE3C0319582906154B
:10029000201C201086150F3086053C08F039860496
:1002A00000008611BC0E0000201849293230BC2104
:1002B0003D08782AA11B0B29080003178D0003179E
:1002C00083168C130C1483120C088D0A782A0317DA
:1002D0008C0083168C130C1555308D00AA308D00C0
:1002E0008C148C1871290C1183128D0A782AA500A0
:1002F000A201250803178D000313260803178F009A
:100300008A210319782A5A21A50A0319A60AA20FDD
:100310007929782A831603178C170C140000000023
:1003200083120C08782ABC00BC0DBC0D3C0D38397A
:1003300041389F002730B1001030BD211F151F1913
:100340009F291E08C30083161E088312C200782A44
:1003500083178001840AFF3E031DA929782AB5016D
:10036000B400FF30B407031CB507031C782A033020
:10037000B100E730BD21B129B101FC3EB000B109A7
:10038000031CC829FF300000B0070318C329B007B9
:100390000000B10FC229080033083B068039BD00B8
:1003A000B31FDD29B009B109B209B309B00A0319B5
:1003B000B10A0319B20A0319B30ABB1FEA29B80923
:1003C000B909BA09BB09B80A0319B90A0319BA0A63
:1003D0000319BB0AB401B501B601B701C601C701D3
:1003E000C801C9013B083A04390438040319282A12
:1003F0002030BC000310B00DB10DB20DB30DC60D11
:10040000C70DC80DC90D3B084902031D112A3A0842
:100410004802031D112A39084702031D112A380812
:100420004602031C222A3808C6023908031C390F69
:10043000C7023A08031C3A0FC8023B08031C3B0FD3
:10044000C9020314B40DB50DB60DB70DBC0BFA29D6
:10045000BD1F352AB409B509B609B709B40A03198D
:10046000B50A0319B60A0319B70A4608B8004708BF
:10047000B9004808BA004908BB003408B000350884
:10048000B1003608B2003708B300782AB901B801C4
:100490001030BC00310DB80DB90D3408B802350864
:1004A000031C350FB90203185C2A3408B807350855
:1004B0000318350FB9070310B00DB10DBC0B4A2A54
:1004C0003008782A1030C100B101B001BD0CBC0C5D
:1004D000031C702A3408B00735080318350FB1071C
:1004E000B10CB00CB90CB80CC10B662A3808782ACC
:1004F0008313831203130000080029082D06D1007E
:10050000D11BB62AA91B9D2A28082C02031C0034E3
:10051000031D013429082D02031C0034031D01347E
:100520002A082E02031C0034031D01342B082F025D
:10053000031C0034031D013400342C082802031C62
:100540000034031D01342D082902031C0034031D4F
:1005500001342E082A02031C0034031D01342F0825
:100560002B02031C0034031D01340034AD1F013481
:1005700000342D082906D100D11BF22AAD1BD92A3F
:100580002C082802031C0034031D01342D08290205
:10059000031C0034031D01342E082A02031C0034FE
:1005A000031D01342F082B02031C0034031D0134EA
:1005B000003428082C02031C0034031D01342908D0
:1005C0002D02031C0034031D01342A082E02031CD3
:1005D0000034031D01342B082F02031C0034031DBB
:1005E00001340034A91F013400342D082906D1003C
:1005F000D11B2A2BAD1B132B2C082802031C003403
:10060000031D01342D082902031C0034031D01348D
:100610002E082A02031C0034031D01342F082B026C
:10062000031C0034013428082C02031C0034031D71
:10063000013429082D02031C0034031D01342A084B
:100640002E02031C0034031D01342B082F02031C4F
:1006500000340134A91F013400342C082802031D82
:1006600000342D082902031D00342E082A02031D20
:1006700000342F082B02031D003401342C08031909
:1006800000348030AD0629082D06D000CD01CE0102
:1006900028082C02031C642B2C08CC002808AC0072
:1006A0004C08A8002D08CC002908AD004C08A90072
:1006B0002E08CC002A08AE004C08AA002F08CC0057
:1006C0002B08AF004C08AB002C0803190034290894
:1006D000D300A917AD172C082802AC000319972BDB
:1006E00008302C02031C8D2BAC002F08CE002E08E6
:1006F000AF002D08AE00AD0108302C02031C8D2B7D
:10070000AC002F08CE002E08AF00AE0108302C023E
:10071000031C8D2B5308A90000342C080319972BB8
:100720000310AD0CAE0CAF0CCE0CAC0B902BD01F4D
:10073000A42BCE09AF09AE09AD09CE0A0319AF0A41
:100740000319AE0A0319AD0A4E08CD072F08031886
:100750002F0FAB072E0803182E0FAA072D0803181A
:100760002D0FA907D01BBD2B031CF62CA90CAA0C1E
:10077000AB0CCD0CA80FF62C362D0318C72CCD09C9
:10078000AB09AA09A909CD0A0319AB0A0319AA0AD8
:100790000319A90A8030D306092D2C080319552CFA
:1007A00028080319442D29082D06D300A917AD17D1
:1007B000D0012908CD002A08CB002B08CC002F0837
:1007C000CC022E08031C2E0FCB022D08031C2D0F6C
:1007D000CD02CD01CB01CC01031CF52B0310A90CDC
:1007E000AA0CAB0CCD0C0130D0002C08A802031CC5
:1007F000FF2B7E305007A8070318362D042C7E30BF
:100800005007A807031C2B2D1830D200CC0DCB0DA0
:10081000CD0DAB0DAA0DA90DD00D2F08AB022E08E2
:10082000031C2E0FAA022D08031C2D0FA9022D0D4B
:10083000D004501C1D2C4C14282C2F08AB072E085C
:1008400003182E0FAA072D0803182D0AA9074C100C
:10085000D20B062C4F1B4C1C4C2C0310AB0DAA0DBD
:10086000A90DD00D2F08AB022E08031C2E0FAA02D3
:100870002D08031C2D0FA9022D0D50040139CC07A2
:100880000318CB0A0319CD0A031D4C2CCD0CCB0C3D
:10089000CC0CA80A0319362DD31FCD134D08A9007F
:1008A0004B08AA004C08AB000034CF15FF342808D1
:1008B000031D2C080319442D29082D06D3002C08EC
:1008C000A8077E30031C682CA8020318362D6B2C59
:1008D000A802031C2B2D2908CD002A08CB002B08C9
:1008E000CC00CD17AD170310A901AA01AB01183038
:1008F000D0004C1C852C2F08AB072E0803182E0F98
:10090000AA072D0803182D0FA907A90CAA0CAB0CD8
:10091000CD0CCB0CCC0C0310D00B792CA91B952C37
:10092000CD0DAB0DAA0DA90DA8034F1B2B1CA72C99
:10093000CD1FA72CAB0A0319AA0A0319A90A031D84
:10094000A72CA90CAA0CAB0CA80A0319362DD31F8F
:10095000A9130034A800A901AA01AB012808CD0001
:100960002B08A8002908AB002808A9009E30A80081
:10097000D301A91FC72CCD09AB09AA09A909CD0A22
:100980000319AB0A0319AA0A0319A90AD317D0013C
:100990002908031DE72C2A08A9002B08AA004D08E6
:1009A000AB00CD01D0152908031DE72C2A08A900AA
:1009B0002B08AA00AB01D01150162908031DE72C03
:1009C0002A08A900AA01D01529080319442D5008A6
:1009D000A802031D031C2B2D0310A91BF62CCD0D03
:1009E000AB0DAA0DA90DA80BED2C2B2D4F1B2B1C0D
:1009F000412DCD1F412DAB0A0319AA0A0319A90ADB
:100A0000031D412DA90CAA0CAB0CA80A0319362D05
:100A1000412DD0012908031D1E2D2A08A9002B08ED
:100A2000AA00AB01D0152908031D1E2D2A08A90014
:100A3000AA01D011501629080319442D5008A80204
:100A4000031D031C2B2D0310A91B412DAB0DAA0D5B
:100A5000A90DA80B242D4F15CF1FFF340130A8007E
:100A6000A901AA01AB01D30DA90CFF34CF14CF1FEC
:100A7000FF34FF30A800A900AA00AB00D30DA90CD9
:100A8000FF34D31FA9130034A901AA01AB01CD0182
:100A9000A8010034BC002408BD003C0824070F2036
:100AA0000008782A6030CF00A001073083169C0030
:100AB00007309F001F3085001F149F141F119F11C6
:100AC0008B170B168312203084005C308A01A92119
:100AD000A030840050308A01A92110308400603099
:100AE0008A01A8219030840060308A01A8218A01FF
:100AF00038208030A10080308A0142201D30A600BD
:100B000023308A0177218030A100C1308A01422040
:100B10001D30A60033308A0177210730B500D03070
:100B20008A01B02100308A015D218316CA0001309C
:100B300083128A015D218316013903193C12031DBA
:100B40003C16023083128A015D2183160139031994
:100B5000BC12031DBC16033083128A015D2183166B
:100B600001390319BC11031DBC15043083128A011D
:100B70005D218316CC00BC103C140130C200013052
:100B8000C6000730C7003C110A30B3008A110A12B0
:100B90008312871FCE2D8A150A1682288A110A12FF
:100BA00083168310BC1D831483128318F22D8A01CF
:100BB00038208030A10080308A0142201D30A600FC
:100BC00042308A0177218030A100C0308A01422062
:100BD0001D30A6004F308A0177210730B500D03094
:100BE0008A01B0218A0138208030A10084308A0136
:100BF00042201D30A6005E308A01772183168512BF
:100C000083128516C8308A01AF218316851283129C
:100C100085128316871083128714C8308A01AF218A
:100C20008316871083128710831607118312071506
:100C3000C8308A01AF21831607118312071183166A
:100C4000871183128715C8308A01AF218316871157
:100C5000831287118316071083120714C8308A0184
:100C6000AF2183160710831207108A150A16542421
:100C70008A110A1611278A0138208A150A12FC21C6
:100C80008A150A12A7218A150A129F228A150A16A6
:100C900054248A110A12831683103C1E8314831273
:100CA0008318592E06308316C70083128A110A1240
:100CB0005C2E04308316C70083125D08AB005C080D
:100CC000AA005B08A9005A08A800CD30AF00CC30BC
:100CD000AE001C30AD008130AC008A01B922CA00E0
:100CE0006108AB006008AA005F08A9005E08A800C0
:100CF000CD30AF00CC30AE001C30AD008130AC0048
:100D00008A01B9224A048A110A1203198E2E831607
:100D10008512831285168A110A12922E8316851265
:100D200083128512031083164A0D8312A700031045
:100D3000A70D01308316C900831283164908831258
:100D400027028A150A12031CA5298A110A12871F75
:100D5000C62E030183163C1901308312CA000430E9
:100D6000831646020130031D003083124A058A11A2
:100D70000A120319BE2E8A150A16C92A8316C60A34
:100D800083128A150A167A208A01382083164608AB
:100D900047028A110A1283120318D12E01308316DA
:100DA000C60083128316B3088A110A128312031D28
:100DB000DC2E07308316C6008312013083164602EC
:100DC0008A110A128312031D722F8A110A16112723
:100DD0008030A10080308A014220831620088312CF
:100DE000C5007B08C4007A08C3007908C20001303E
:100DF0008A017B2020308A010B218316250883126B
:100E00008A010B211D30A60067308A0177218030CE
:100E1000A1008C308A0142200530A500B901BD3007
:100E20008A01FB208030A100C0308A014220740872
:100E3000C5007308C4007208C3007108C200013005
:100E40008A017B201D30A60071308A017721AB0119
:100E5000AA014030A9008130A8008316320883120D
:100E6000AF00831631088312AE0083163008831258
:100E7000AD0083162F088312AC008A012D23013C9C
:100E80008A110A12031D512F8030A100CA308A0135
:100E900042201D30A60078308A0177218A110A127B
:100EA000722F8030A100CA308A01422020308A018E
:100EB0000B2131308A010B213A308A010B21831634
:100EC00032088312C500831631088312C4008316CA
:100ED00030088312C30083162F088312C20001302A
:100EE0008A017B200230831646028A110A1283127D
:100EF000031DE62F8030A10080308A014220463059
:100F00008A010B2157308A010B2144308A010B21C1
:100F10003A308A010B2120308A010B2183162008E8
:100F20008312C5007B08C4007A08C3007908C20098
:100F300001308A017B2020308A010B21831625088D
:100F400083128A010B2157308A010B2120308A013C
:100F50000B218A010B218A010B218030A100C030B6
:100F60008A01422052308A010B2145308A010B212F
:100F700046308A010B213A308A010B2120308A0148
:100F80000B21831624088312C500831623088312BD
:100F9000C400831622088312C3008316210883121B
:100FA000C20001308A017B2020308A010B21831688
:100FB000260883128A010B2157308A010B21203029
:100FC0008A010B218A010B218A010B210330831630
:100FD00046028A150A128312031D36288030A100AA
:100FE00080308A01422046308A010B2157308A0125
:100FF0000B2144308A010B213A308A010B21203029
:101000008A010B217408C5007308C4007208C3006C
:101010007108C20001308A017B201D30A6007F309C
:101020008A0177218030A100C0308A0142205230ED
:101030008A010B2145308A010B2146308A010B21A0
:101040003A308A010B2120308A010B217808C50033
:101050007708C4007608C3007508C20001308A0111
:101060007B201D30A60086308A017721043083164C
:1010700046028A150A128312031D6E288030A100D1
:1010800080308A0142201D30A6008D308A017721F0
:101090008A150A12831683103C1D83148312831849
:1010A0005B288030A100C3308A0142201D30A60099
:1010B0009E308A0177218A150A12831683103C1903
:1010C0008314831283186E288030A100C3308A01F4
:1010D00042201D30A600A8308A01772105308316F2
:1010E00046028A150A128312031DF0288030A100DF
:1010F00080308A01422046308A010B213A308A0131
:101100000B2120308A010B215D08C5005C08C4005A
:101110005B08C3005A088A150A12031D90284F1550
:101120008A150A12031995285A03C20002308A014F
:101130007B2056308A010B2120308A010B21283078
:101140008A010B21A601831628088312B900831691
:1011500027088312B8008A014C2029308A010B210C
:1011600020308A010B218030A100C0308A0142204A
:1011700052308A010B213A308A010B2120308A013A
:101180000B216108C5006008C4005F08C3005E0849
:101190008A150A12031DCD284F158A150A12031944
:1011A000D2285E03C20002308A017B2056308A01B9
:1011B0000B2120308A010B2128308A010B21A60146
:1011C00083162A088312B900831629088312B800EF
:1011D0008A014C2029308A010B2120308A010B2101
:1011E0000630831646028A150A128312031D4A2905
:1011F0008A110A1611278030A10080308A0142200E
:101200001D30A600B2308A0177218030A100C030A5
:101210008A01422046308A010B213A308A010B2193
:10122000831637088312C500831636088312C4005C
:10123000831635088312C300831634088312C20054
:1012400001308A017B2020308A010B2152308A0133
:101250000B213A308A010B2183163B088312C5000B
:1012600083163A088312C400831639088312C30018
:10127000831638088312C20001308A017B20803037
:10128000A1008C308A0142200530A500B901BD3093
:101290008A01FB200730831646028A150A12831240
:1012A000031D9E298A110A1611278030A100803063
:1012B0008A014220831620088312C5007B08C400DF
:1012C0007A08C3007908C20001308A017B202030EF
:1012D0008A010B218316250883128A010B211D30F8
:1012E000A600BD308A0177218030A1008C308A01B0
:1012F00042200530A500B901BD308A01FB208030B5
:10130000A100C0308A0142207408C5007308C400DF
:101310007208C3007108C20001308A017B201D30B1
:10132000A600C7308A0177218030A100CA308A0127
:1013300042201D30A600CE308A0177218316C90ACB
:101340008A110A128312031D9C2E8A013D2E003041
:101350008A019321D4004308D50055088316A800BC
:10136000831254088316A70083128A150A12572283
:101370006C08AB006B08AA006A08A9006908A800FD
:10138000831637088312AF00831636088312AE0027
:10139000831635088312AD00831634088312AC001F
:1013A0008A0143232B08EC002A08EB002908EA00F5
:1013B0002808E9008A150A12D0266C08F4006B0888
:1013C000F3006A08F2006908F10065088316A000BE
:1013D00083126408FB006308FA006208F9006608DB
:1013E0008316A50083125908DD005808DC00570851
:1013F000DB005608DA00080001308A019321D4008E
:101400004308D50055088316AA0083125408831692
:10141000A90083128A150A1257226C08AB006B08C8
:10142000AA006A08A9006908A80083163B0883126D
:10143000AF0083163A088312AE0083163908831270
:10144000AD00831638088312AC008A0143232B08B1
:10145000EC002A08EB002908EA002808E9008A15B0
:101460000A12D0266C08F8006B08F7006A08F6002C
:101470006908F50065088316A400831264088316C2
:10148000A300831263088316A200831262088316E6
:10149000A100831266088316A60083125908E10092
:1014A0005808E0005708DF005608DE000800AF01CA
:1014B0009830AE004C30AD008C30AC005508A9001F
:1014C0005408A8008A01AC248A01CD232B08D90036
:1014D0002A08D8002908D7002808D600AB01AA019D
:1014E0002030A9008330A8005908AF005808AE008A
:1014F0005708AD005608AC008A0157242B08C500D8
:101500002A08C4002908C3002808C200AF01AE01A0
:101510003430AD008530AC004508AB004408AA006B
:101520004308A9004208A8008A013E232B08EC00CA
:101530002A08EB002908EA002808E90008007408D6
:10154000AB007308AA007208A9007108A800780807
:10155000AF007708AE007608AD007508AC008A01D0
:101560003E232B088316AE0083122A088316AD0093
:10157000831229088316AC00831228088316AB0057
:10158000B201B1014030B0008130AF00AB088A1524
:101590000A1283120319DA2A8A150A128316831093
:1015A000AC1F831483128318DA2A8316AE01AD01AF
:1015B000AC01AB018312AB01AA016030A9008030FD
:1015C000A80083162E088312AF0083162D088312FD
:1015D000AE0083162C088312AD0083162B088312ED
:1015E000AC008A01F522013C8A150A120319FF2A70
:1015F0008316B201B1012030B0008130AF008312F8
:10160000CD30AB00CC30AA000C30A9008130A8004E
:1016100083162E088312AF0083162D088312AE00A6
:1016200083162C088312AD0083162B088312AC009E
:101630008A01F522013C8A150A120319252B83160B
:10164000B201B101B0018130AF008312CD30AB00E7
:10165000CC30AA001C30A9008130A80083162E08C7
:101660008312AF0083162D088312AE0083162C0858
:101670008312AD0083162B088312AC008A01F52279
:10168000013C8A150A1203194C2B66308316B200EE
:10169000B100B0008030AF0083126630AB00AA000A
:1016A0002630A9008130A80083162E088312AF00CF
:1016B00083162D088312AE0083162C088312AD000A
:1016C00083162B088312AC008A01F522013C8A158F
:1016D0000A120319742B9A308316B2009930B100A4
:1016E0005930B0008030AF008312AB01AA01403006
:1016F000A9008130A80083162E088312AF0083163C
:101700002D088312AE0083162C088312AD008316B9
:101710002B088312AC008A01F522013C8A150A12BB
:101720000319992B8316B201B1014030B00080300B
:10173000AF008312CD30AB00CC30AA004C30A900F2
:101740008130A80083162E088312AF0083162D085F
:101750008312AE0083162C088312AD0083162B086B
:101760008312AC008A01F522013C8A150A12031982
:10177000C02B33308316B200B100B0008030AF0010
:101780008312AB01AA016030A9008130A800831642
:101790002E088312AF0083162D088312AE00831625
:1017A0002C088312AD0083162B088312AC008A012B
:1017B000F522013C8A150A120319E62B66308316BE
:1017C000B200B1002630B0008030AF008312663026
:1017D000AB00AA007630A9008130A80083162E083D
:1017E0008312AF0083162D088312AE0083162C08D7
:1017F0008312AD0083162B088312AC008A01F522F8
:10180000013C8A150A1203190E2C9A308316B20075
:101810009930B1001930B0008030AF008312AB01B5
:10182000AA010830A9008230A80083162E0883126E
:10183000AF0083162D088312AE0083162C08831286
:10184000AD0083162B088312AC008A01F522013CFF
:101850008A150A120319352CCD308316B200CC300C
:10186000B1000C30B0008030AF008312AB01AA0190
:101870001830A9008230A80083162E088312AF000A
:1018800083162D088312AE0083162C088312AD0038
:1018900083162B088312AC008A01F522013C8A15BD
:1018A0000A120319592C8316B201B101B00180301C
:1018B000AF0083129A30AB009930AA002130A90002
:1018C0008230A80083162E088312AF0083162D08DD
:1018D0008312AE0083162C088312AD0083162B08EA
:1018E0008312AC008A01F522013C8A150A12031901
:1018F000812C33308316B200B1007330B0007F30DA
:10190000AF008312CD30AB00CC30AA002C30A90040
:101910008230A80083162E088312AF0083162D088C
:101920008312AE0083162C088312AD0083162B0899
:101930008312AC008A01F522013C8A150A120319B0
:10194000A82C66308316B200B100B0007F30AF0023
:1019500083123330AB00AA003B30A9008230A800CC
:1019600083162E088312AF0083162D088312AE0053
:1019700083162C088312AD0083162B088312AC004B
:101980008A01F522013C8A150A120319D02C9A30DB
:101990008316B2009930B1005930B0007F30AF00EB
:1019A00083123330AB00AA004B30A9008230A8006C
:1019B00083162E088312AF0083162D088312AE0003
:1019C00083162C088312AD0083162B088312AC00FB
:1019D0008A01F522013C8A150A120319F82CCD3030
:1019E0008316B200CC30B1004C30B0007F30AF0075
:1019F00083126630AB00AA005E30A9008230A800D6
:101A000083162E088312AF0083162D088312AE00B2
:101A100083162C088312AD0083162B088312AC00AA
:101A20008A01F522013C8A150A1203191E2D83161C
:101A3000B201B1014030B0007F30AF008312AB0182
:101A4000AA017830A9008230A80083162E088312DC
:101A5000AF0083162D088312AE0083162C08831264
:101A6000AD0083162B088312AC008A01F522013CDD
:101A70008A150A120319432D33308316B200B100C0
:101A8000B0007F30AF0083129A30AB009930AA00CB
:101A90000D30A9008330A80083162E088312AF00F2
:101AA00083162D088312AE0083162C088312AD0016
:101AB00083162B088312AC008A01F522013C8A159B
:101AC0000A1203196B2D66308316B200B10026305E
:101AD000B0007F30AF0083126630AB00AA00263022
:101AE000A9008330A80083162E088312AF00831646
:101AF0002D088312AE0083162C088312AD008316C6
:101B00002B088312AC008A01F522013C8A150A12C7
:101B10000319932D9A308316B2009930B100193011
:101B2000B0007F30AF0083123330AB00AA005330D7
:101B3000A9008330A80083162E088312AF008316F5
:101B40002D088312AE0083162C088312AD00831675
:101B50002B088312AC008A01F522013C8A150A1277
:101B60000319BB2DCD308316B200CC30B1000C3040
:101B7000B0007F30AF008312AB01AA017030A90022
:101B80008330A80083162E088312AF0083162D0819
:101B90008312AE0083162C088312AD0083162B0827
:101BA0008312AC008A01F522013C8A150A1203193E
:101BB000DF2D8316B201B101B0017F30AF00831277
:101BC0000230831633020130031D00308312CA0035
:101BD00003018316BC1A013083124A058A150A12C2
:101BE0000319CF2E9A30AB009930AA005930A900C2
:101BF0007F30A800831632088312AF0083163108A5
:101C00008312AE00831630088312AD0083162F08AE
:101C10008312AC008A012D23CA0083163208831276
:101C2000AB00831631088312AA0083163008831292
:101C3000A90083162F088312A8009A30AF009930AC
:101C4000AE005930AD007F30AC008A017D224A04DD
:101C50008A150A120319352ECD308316B200CC3006
:101C6000B1000C30B0007F30AF0083126630AB00A3
:101C7000AA00A9007F30A800831632088312AF00A3
:101C8000831631088312AE00831630088312AD002C
:101C900083162F088312AC008A012D23013C8A157C
:101CA0000A12031D5B2E66308316B200B100263087
:101CB000B0007F30AF0083123330AB00AA00733026
:101CC000A9007F30A800831632088312AF00831664
:101CD00031088312AE00831630088312AD008316DC
:101CE0002F088312AC008A012D23013C8A150A12A9
:101CF000031D812E8316B201B1014030B0007F3048
:101D0000AF008312AB01AA01A9018030A80083169D
:101D100032088312AF00831631088312AE00831697
:101D200030088312AD0083162F088312AC008A019D
:101D30002D23013C8A150A12031DA72E9A30831603
:101D4000B2009930B1005930B0007F30AF0083123B
:101D50006630AB00AA000630A9008030A8008316C8
:101D600032088312AF00831631088312AE00831647
:101D700030088312AD0083162F088312AC008A014D
:101D80002D23013C8A150A12031DCE2E33308316F3
:101D9000B200B1007330B0007F30AF008312080092
:101DA0006C08AB006B08AA006A08A9006908A800C3
:101DB000AF01AE01CC30AD008430AC008A01F52219
:101DC000013C8A150A120319EB2EEC01EB01CC3011
:101DD000EA008430E9006C08AB006B08AA006A08CE
:101DE000A9006908A800AF01AE01C830AD00843079
:101DF000AC008A01F522013C8A150A120319202F32
:101E0000AB01AA017030A9008430A8006C08AF00B3
:101E10006B08AE006A08AD006908AC008A01432374
:101E20002B08F0002A08EF002908EE002808ED0032
:101E3000E8010130E7006E30E6008A110A164B29EE
:101E40006C08AB006B08AA006A08A9006908A80022
:101E5000AF01AE01A030AD008430AC008A01F522A4
:101E6000013C8A150A120319552FAB01AA0148300B
:101E7000A9008430A8006C08AF006B08AE006A08A7
:101E8000AD006908AC008A0143232B08F0002A0842
:101E9000EF002908EE002808ED00E8010A30E7000D
:101EA0006E30E6008A110A164B296C08AB006B08ED
:101EB000AA006A08A9006908A800AF01AE01F030C5
:101EC000AD008330AC008A01F522013C8A150A126C
:101ED00003198A2FAB01AA012030A9008430A80081
:101EE0006C08AF006B08AE006A08AD006908AC0072
:101EF0008A0143232B08F0002A08EF002908EE008E
:101F00002808ED00E8016430E7006E30E6008A1131
:101F10000A164B296C08AB006B08AA006A08A900D6
:101F20006908A800AF01AE01A030AD008330AC005D
:101F30008A01F522013C8A150A120319BF2FAB0151
:101F4000AA017030A9008330A8006C08AF006B08AC
:101F5000AE006A08AD006908AC008A0143232B0873
:101F6000F0002A08EF002908EE002808ED00E8013B
:101F70000130E7007530E6008A110A164B296C081B
:101F8000AB006B08AA006A08A9006908A800AF01A5
:101F9000AE01A030AD008230AC008A01F522013CD8
:101FA0008A150A120319F42FAB01AA012030A900E7
:101FB0008330A8006C08AF006B08AE006A08AD0063
:101FC0006908AC008A0143232B08F0002A08EF00BF
:101FD0002908EE002808ED00E8010A30E700753016
:101FE000E6008A110A164B29E9088A110A16031914
:101FF0001D288A110A16EA1F1D28AB01AA012030EC
:10200000A9008230A8006C08AF006B08AE006A0817
:10201000AD006908AC008A0143232B08F0002A08B0
:10202000EF002908EE002808ED00E8016430E70021
:102030007530E6008A110A164B296C08AB006B0854
:10204000AA006A08A9006908A800AF01AE01203003
:10205000AD008230AC008A01F522013C8A110A16DB
:10206000031942286C08F0006B08EF006A08EE00C4
:102070006908ED00E8010130E7006D30E6008A11E3
:102080000A164B296C08AB006B08AA006A08A90065
:102090006908A800AF01AE012030AD008330AC006C
:1020A0008A01F522013C8A110A1603197728AF012B
:1020B000AE012030AD008230AC006C08AB006B0884
:1020C000AA006A08A9006908A8008A013E232B0813
:1020D000F0002A08EF002908EE002808ED00E801CA
:1020E0000A30E7006D30E6008A110A164B296C08A9
:1020F000AB006B08AA006A08A9006908A800AF0134
:10210000AE017030AD008330AC008A01F522013C95
:102110008A110A160319AC28AF01AE012030AD00B8
:102120008330AC006C08AB006B08AA006A08A900F9
:102130006908A8008A013E232B08F0002A08EF0056
:102140002908EE002808ED00E8016430E7006D3052
:10215000E6008A110A164B296C08AB006B08AA002E
:102160006A08A9006908A800AF01AE012030AD00DF
:102170008430AC008A01F522013C8A110A16031949
:10218000E128AF01AE017030AD008330AC006C08C7
:10219000AB006B08AA006A08A9006908A8008A01B8
:1021A0003E232B08F0002A08EF002908EE0028083B
:1021B000ED00E8010130E7002030E6008A110A1640
:1021C0004B296C08AB006B08AA006A08A9006908D3
:1021D000A800AF01AE014830AD008430AC008A01E8
:1021E000F522013C8A110A1603191629AF01AE0126
:1021F0002030AD008430AC006C08AB006B08AA0046
:102200006A08A9006908A8008A013E232B08F0008B
:102210002A08EF002908EE002808ED00E8010A303E
:10222000E7002030E6008A110A164B296C08AB0043
:102230006B08AA006A08A9006908A800AF01AE01EE
:102240007030AD008430AC008A01F522013C8A1167
:102250000A1603194B29AF01AE014830AD00843096
:10226000AC006C08AB006B08AA006A08A9006908FA
:10227000A8008A013E232B08F0002A08EF00290855
:10228000EE002808ED00E8016430E7002030E600A9
:102290008A110A164B29AB01AA01A901A8017008ED
:1022A000AF006F08AE006E08AD006D08AC008A018B
:1022B000B922013C8A110A1603196329E501E401D8
:1022C000E3017F30E2003330AB00AA00A9007E308A
:1022D000A8007008AF006F08AE006E08AD006D0872
:1022E000AC008A01F522013C8A110A1603198029E3
:1022F0009A30E5009930E4001930E3007F30E200C5
:102300003330AB00AA00A9007F30A8007008AF00EE
:102310006F08AE006E08AD006D08AC008A01F522B2
:10232000013C8A110A1603199B293330E500E400A9
:10233000E3007F30E2003330AB00AA007330A90025
:102340007F30A8007008AF006F08AE006E08AD00C7
:102350006D08AC008A01F522013C8A110A160319A6
:10236000B929CD30E500CC30E4004C30E3007F30BB
:10237000E2009A30AB009930AA001930A9008030F1
:10238000A8007008AF006F08AE006E08AD006D08C1
:10239000AC008A01F522013C8A110A160319D629DC
:1023A0006630E500E400E3007F30E2006630AB0019
:1023B000AA002630A9008030A8007008AF006F087E
:1023C000AE006E08AD006D08AC008A01F522013C3C
:1023D0008A110A160319F3293330E500E40073303B
:1023E000E3007F30E200AB01AA014030A900803059
:1023F000A8007008AF006F08AE006E08AD006D0851
:10240000AC008A01F522013C8A110A1603190D2A33
:10241000E501E401E3018030E2009A30AB0099303D
:10242000AA005930A9008030A8007008AF006F08DA
:10243000AE006E08AD006D08AC008A01F522013CCB
:102440008A110A1603192C2ACD30E500CC30E4009D
:102450000C30E3008030E2006630AB00AA00A90037
:102460008030A8007008AF006F08AE006E08AD00A5
:102470006D08AC008A01F522013C8A110A16031985
:10248000482A3330E500E4001330E3008030E200F6
:102490009A30AB009930AA007930A9008030A800AA
:1024A0007008AF006F08AE006E08AD006D08AC009C
:1024B0008A01F522013C8A110A160319652AE501F1
:1024C000E4012030E3008030E200CD30AB00CC30BE
:1024D000AA000C30A9008130A8007008AF006F0876
:1024E000AE006E08AD006D08AC008A01F522013C1B
:1024F0008A110A160319822A3330E500E400E3004A
:102500008030E2003330AB00AA001330A9008130E4
:10251000A8007008AF006F08AE006E08AD006D082F
:10252000AC008A01F522013C8A110A1603199E2A81
:10253000E501E4014030E3008030E200CD30AB0043
:10254000CC30AA001C30A9008130A8007008AF0070
:102550006F08AE006E08AD006D08AC008A01F52270
:10256000013C8A110A160319BD2ACD30E500CC3092
:10257000E4004C30E3008030E200CD30AB00CC30E2
:10258000AA002C30A9008130A8007008AF006F08A5
:10259000AE006E08AD006D08AC008A01F522013C6A
:1025A0008A110A160319DA2AE501E4016030E30012
:1025B0008030E2006630AB00AA003630A9008130DE
:1025C000A8007008AF006F08AE006E08AD006D087F
:1025D000AC008A01F522013C8A110A160319F72A78
:1025E0003330E500E4007330E3008030E200CD30AA
:1025F000AB00CC30AA003C30A9008130A8007008A4
:10260000AF006F08AE006E08AD006D08AC008A0127
:10261000F522013C8A110A160319132BE501E40186
:10262000E3018130E2006630AB00AA004630A90029
:102630008130A8007008AF006F08AE006E08AD00D2
:102640006D08AC008A01F522013C8A110A160319B3
:10265000302B6630E500E4000630E3008130E20014
:10266000CD30AB00CC30AA004C30A9008130A8009E
:102670007008AF006F08AE006E08AD006D08AC00CA
:102680008A01F522013C8A110A1603194D2BE50136
:10269000E4011030E3008130E2003330AB00AA00E7
:1026A0005330A9008130A8007008AF006F08AE0059
:1026B0006E08AD006D08AC008A01F522013C8A115C
:1026C0000A1603196A2B6630E500E4001630E300B1
:1026D0008130E200CD30AB00CC30AA005C30A900E4
:1026E0008130A8007008AF006F08AE006E08AD0022
:1026F0006D08AC008A01F522013C8A110A16031903
:10270000872BE501E4012030E3008130E2006630F0
:10271000AB00AA00A9008130A8007008AF006F08C4
:10272000AE006E08AD006D08AC008A01F522013CD8
:102730008A110A160319A42BCD30E500CC30E40031
:102740002C30E3008130E200CD30AB00CC30AA0069
:102750006C30A9008130A8007008AF006F08AE008F
:102760006E08AD006D08AC008A01F522013C8A11AB
:102770000A160319C12B3330E500E400E300813071
:10278000E2003330AB00AA007330A9008130A8000A
:102790007008AF006F08AE006E08AD006D08AC00A9
:1027A0008A01F522013C8A110A160319DF2BCD306C
:1027B000E500CC30E4003C30E3008130E200CD3075
:1027C000AB00CC30AA007C30A9008130A800700892
:1027D000AF006F08AE006E08AD006D08AC008A0156
:1027E000F522013C8A110A160319FE2B9A30E500E6
:1027F0009930E4004930E3008130E2003330AB002F
:10280000AA000330A9008230A8007008AF006F084A
:10281000AE006E08AD006D08AC008A01F522013CE7
:102820008A110A1603191C2C9A30E5009930E4002D
:102830005930E3008130E2006630AB00AA00063078
:10284000A9008230A8007008AF006F08AE006E08C3
:10285000AD006D08AC008A01F522013C8A110A1610
:102860000319382CE501E4016030E3008130E20017
:102870009A30AB009930AA000930A9008230A80034
:102880007008AF006F08AE006E08AD006D08AC00B8
:102890008A01F522013C8A110A160319552C66306B
:1028A000E500E400E3008130E2003330AB00AA0031
:1028B0000B30A9008230A8007008AF006F08AE008E
:1028C0006E08AD006D08AC008A01F522013C8A114A
:1028D0000A160319712CE501E4017030E300813020
:1028E000E200CD30AB00CC30AA000C30A900823021
:1028F000A8007008AF006F08AE006E08AD006D084C
:10290000AC008A01F522013C8A110A1603198F2CAA
:102910006630E500E4007630E3008130E2006630A6
:10292000AB00AA000E30A9008230A8007008AF00EA
:102930006F08AE006E08AD006D08AC008A01F5228C
:10294000013C8A110A160319AA2CE501E401E301EE
:102950008230E2009A30AB009930AA001130A90011
:102960008230A8007008AF006F08AE006E08AD009E
:102970006D08AC008A01F522013C8A110A16031980
:10298000C92CCD30E500CC30E4000430E3008230C7
:10299000E2003330AB00AA001330A9008230A80057
:1029A0007008AF006F08AE006E08AD006D08AC0097
:1029B0008A01F522013C8A110A160319E52CE5016A
:1029C000E4010830E3008230E200CD30AB00CC30CF
:1029D000AA001430A9008230A8007008AF006F0868
:1029E000AE006E08AD006D08AC008A01F522013C16
:1029F0008A110A160319032D6630E500E4000E3033
:102A0000E3008230E2006630AB00AA001630A90075
:102A10008230A8007008AF006F08AE006E08AD00ED
:102A20006D08AC008A01F522013C8A110A160319CF
:102A30001F2DE501E4011030E3008230E200AB011C
:102A4000AA011830A9008230A8007008AF006F08F2
:102A5000AE006E08AD006D08AC008A01F522013CA5
:102A60008A110A1603193C2D9A30E5009930E400CA
:102A70001130E3008230E2009A30AB009930AA00B6
:102A80001930A9008230A8007008AF006F08AE00AE
:102A90006E08AD006D08AC008A01F522013C8A1178
:102AA0000A1603195B2DCD30E500CC30E40014305C
:102AB000E3008230E2003330AB00AA001B30A900F3
:102AC0008230A8007008AF006F08AE006E08AD003D
:102AD0006D08AC008A01F522013C8A110A1603191F
:102AE000792D9A30E5009930E4001930E300823006
:102AF000E200CD30AB00CC30AA001C30A9008230FF
:102B0000A8007008AF006F08AE006E08AD006D0839
:102B1000AC008A01F522013C8A110A160319982D8E
:102B2000CD30E500CC30E4001C30E3008230E20020
:102B30006708A8006808A9008A01AC246508AF00EE
:102B40006408AE006308AD006208AC008A01572437
:102B50002B08E5002A08E4002908E3002808E20021
:102B6000AB01C030AA007930A9008830A800650800
:102B7000AF006408AE006308AD006208AC008A01D3
:102B8000F522013C8A110A160319CD2DE501C0304A
:102B9000E4007930E3008830E20008008A110A1668
:102BA000061CA12E0130831646020130031D0030A1
:102BB0008312CA000630831646020130031D00301E
:102BC00083124A04CA000730831646020130031DEF
:102BD000003083124A048A110A160319FC2D8A1147
:102BE0000A16861CF92D8316C20A83128A110A1648
:102BF000FB2D8316C20383128316C6088A110A1698
:102C00008312031D902E0130831648028A110A1682
:102C10008312031D182E8A110A16861C152E831680
:102C2000CA0A83128A110A16172E8316CA03831240
:102C30000230831648028A110A168312031D392EA8
:102C40008A110A16861C302E831083163C1E8314AC
:102C500083183C16831C3C1283128A110A16382EE4
:102C6000831083163C1E831483183C16831C3C126D
:102C700083120330831648028A110A168312031D39
:102C80005A2E8A110A16861C512E83108316BC1EDA
:102C900083148318BC16831CBC1283128A110A1673
:102CA000592E83108316BC1E83148318BC16831CF4
:102CB000BC1283120430831648028A110A1683124A
:102CC000031D7B2E8A110A16861C722E8310831612
:102CD000BC1D83148318BC15831CBC1183128A117C
:102CE0000A167A2E83108316BC1D83148318BC1514
:102CF000831CBC1183120530831648028A110A1600
:102D00008312031D902E8A110A16861C8D2E83169F
:102D1000CC0A83128A110A168F2E8316CC038312D3
:102D20000430831646028A110A168312031DA02E50
:102D3000831083163C1D831483183C15831C3C119F
:102D400083128316420844020130031803018312E0
:102D5000CA0001308316BC18030183124A058A1188
:102D60000A160319B62E83164408C200831283166E
:102D7000430842020130031803018312CA000130E4
:102D80008316BC18030183124A058A110A16031917
:102D9000CC2E83164308C2008312831642084402D5
:102DA0000130031803018312CA0003018316BC1803
:102DB000013083124A058A110A160319E92E831677
:102DC0004308C20083103C1C831483183C14831CEA
:102DD0003C1083128316430842020130031803019A
:102DE0008312CA0003018316BC18013083124A05FE
:102DF0008A110A160319062F83164408C20083108D
:102E00003C1C831483183C14831C3C1083128B10CD
:102E10007D088A007C0884007E088300FF0E7F0EF8
:102E20000900BD01831642088312BC00B5010D30B4
:102E3000B4008A0162228316C500450883128A0104
:102E40005D218316CD0001304D028A110A168312CE
:102E5000031D342F31308316BD003630BE003030B4
:102E6000BF006D30C000C1018312023083164D02D5
:102E70008A110A168312031D472F20308316BD00C6
:102E80003830BE003030BF006D30C000C101831249
:102E9000033083164D028A110A168312031D5A2F1E
:102EA00020308316BD003430BE003030BF006D309E
:102EB000C000C1018312043083164D028A110A1624
:102EC0008312031D6D2F20308316BD003330BE00EA
:102ED0003030BF006D30C000C10183120530831651
:102EE0004D028A110A168312031D802F203083168B
:102EF000BD003230BE003030BF006D30C000C101B7
:102F00008312063083164D028A110A168312031D9E
:102F1000932F20308316BD003130BE003730BF0004
:102F20006D30C000C1018312073083164D028A1133
:102F30000A168312031DA62F20308316BD003130E0
:102F4000BE003530BF006D30C000C10183120830B3
:102F500083164D028A110A168312031DB92F2030E1
:102F60008316BD003130BE003230BF006D30C0006E
:102F7000C1018312093083164D028A110A16831289
:102F8000031DCC2F20308316BD003130BE00303001
:102F9000BF006D30C000C10183120A3083164D029C
:102FA0008A110A168312031DDE2F20308316BD00FE
:102FB000BE003630BF006D30C000C10183120B303F
:102FC00083164D028A110A168312031DF02F20303A
:102FD0008316BD00BE003230BF006D30C000C1019D
:102FE00083120C3083164D028A150A168312031DB4
:102FF000032837308316BD003030BE006330BF0079
:103000006D30C000C10183120D3083164D028A1548
:103010000A168312031D162832308316BD00333082
:10302000BE006330BF006D30C000C10183120E309E
:1030300083164D028A150A168312031D2928313082
:103040008316BD003330BE006330BF006D30C0005A
:10305000C10183128316B3088A150A168312031D51
:103060004C2809308316450783128A015D21831697
:10307000B40083128A015F218316B50083128A018E
:103080005F218316B60083128A015F218316B70081
:1030900083128A150A1678288316450A83128A0134
:1030A0005D218316B40083128A015F218316B50067
:1030B00083128A015F218316B60083128A015F2181
:1030C0008316B7000530450783128A015D218316F8
:1030D000B80083128A015F218316B90083128A0126
:1030E0005F218316BA0083128A015F218316BB0019
:1030F000831208008A150A16871F81288A150A1666
:103100007A2808008A0138208030A10080308A01A6
:1031100042201D30A600D5308A0177218A150A1673
:103120007A208A0138208316BC14043083128A0165
:103130005D218316CC0083128A150A1654248A1145
:103140000A1611278A150A12A7218A150A12FC21CC
:103150005D08AB005C08AA005B08A9005A08A8003B
:10316000CD30AF00CC30AE001C30AD008130AC00B3
:103170008A01B922CA006108AB006008AA005F0892
:10318000A9005E08A800CD30AF00CC30AE001C30E6
:10319000AD008130AC008A01B9224A048A150A16B2
:1031A0000319D92883168512831285168A150A16E3
:1031B000DD2883168512831285128316B3088A15BB
:1031C0000A168312031DF4288030A10080308A0182
:1031D00042201D30A600E2308A0177218316CC01FF
:1031E00083128A150A1607298030A10080308A01CF
:1031F000422083164C0883128A01492064308A01D8
:103200000B2142308A010B216D308A010B218A1576
:103210000A16831683103C1C8314831283181E29FC
:103220008030A10087308A01422046308A010B217C
:1032300057308A010B2144308A010B218A150A1666
:10324000831683103C188314831283183529803029
:10325000A10087308A01422052308A010B2145307B
:103260008A010B2146308A010B218030A1008C306D
:103270008A0142200530A500B901BD308A01FB203A
:103280008316B3088A150A168312031D5429803049
:10329000A10085308A0142201D30A600E9308A0154
:1032A000772183163C14CC0183128A150A168316E3
:1032B00083103C1C83148312831889298030A10059
:1032C000C0308A0142201D30A600F0308A017721EB
:1032D000831637088312C500831636088312C4008C
:1032E000831635088312C300831634088312C20084
:1032F00001308A017B2020308A010B2164308A0151
:103300000B2142308A010B2120308A010B218A01D6
:103310000B218A150A16831683103C188314831216
:103320008318BD298030A100C0308A0142201D30A1
:10333000A600F7308A01772183163B088312C50067
:1033400083163A088312C400831639088312C30017
:10335000831638088312C20001308A017B20203096
:103360008A010B2164308A010B2142308A010B2132
:1033700020308A010B218A010B218A150A16871F2A
:10338000C62A8A150A16831683103C1C83148312DE
:1033900083180D2A8A150A12A7217408AB00730836
:1033A000AA007208A9007108A800831637088312C2
:1033B000AF00831636088312AE00831635088312D9
:1033C000AD00831634088312AC008A013E232B081B
:1033D000F4002A08F3002908F2002808F1008316F7
:1033E0004C0883128A01AA247408AF007308AE0047
:1033F0007208AD007108AC008A013E232B088316C9
:10340000B70083122A088316B60083122908831690
:10341000B500831228088316B40083128A150A1691
:10342000831683103C188314831283185A2A8A1532
:103430000A12FC217808AB007708AA007608A900D8
:103440007508A80083163B088312AF0083163A085C
:103450008312AE00831639088312AD008316380834
:103460008312AC008A013E232B08F8002A08F700DB
:103470002908F6002808F50083164C0883128A01F3
:10348000AA247808AF007708AE007608AD0075086A
:10349000AC008A013E232B088316BB0083122A0846
:1034A0008316BA00831229088316B90083122808EC
:1034B0008316B80083128316B3088A150A1683127E
:1034C000031D802A093083164507831203178D00D8
:1034D00083160313340883128A0167218316350883
:1034E00083128A0167218316360883128A016721B5
:1034F0008316370883128A0167218A150A16B52AAE
:103500008316450A831203178D00831603133408AC
:1035100083128A0167218316350883128A01672185
:103520008316360883128A016721831637088312AF
:103530008A016721053083164507831203178D0022
:1035400083160313380883128A016721831639080A
:1035500083128A01672183163A0883128A01672140
:1035600083163B0883128A0167218030A100C03096
:103570008A0142201D30A600FE308A0177210330E7
:10358000B500E8308A01B0218A0138208A150A1670
:1035900093288A0138208A150A167A208316C601D4
:1035A0000130C8003C1183128A150A16871FE82AC9
:1035B0008316C80A073048028A150A168312031DAB
:1035C000E32A8A013D2E8A150A167A208A013820BC
:1035D000013083164A028A150A1683120318F32A49
:1035E00001308316CA008312653083164A028A1599
:1035F0000A168312031CFF2A64308316CA00831242
:1036000083164C0A8A150A168312031D092B83168A
:10361000CC0183123D3083164C028A150A168312A0
:10362000031C152B3C308316CC008312013083160B
:1036300048028A150A168312031D3F2B8030A10011
:1036400080308A0142201E30A6000E308A01772188
:103650008030A100C0308A01422083164A088312BC
:103660008A0149201E30A6001F308A0177210317E6
:103670008D01831603134A0883128A0167210230E1
:10368000831648028A150A168312031D822B803086
:10369000A10080308A0142201E30A60029308A0114
:1036A00077218A150A16831683103C1E8314831211
:1036B0008318642B8030A100C3308A0142201E3061
:1036C000A60037308A0177218A150A1683168310DF
:1036D0003C1A831483128318772B8030A100C330E7
:1036E0008A0142201E30A60041308A017721013034
:1036F00003178D000301831603133C1A0130831254
:103700008A0167210330831648028A150A1683123C
:10371000031DC52B8030A10080308A0142201E305D
:10372000A6004B308A0177218A150A16831683106A
:10373000BC1E831483128318A72B8030A100C330D2
:103740008A0142201E30A6005C308A0177218A154A
:103750000A1683168310BC1A831483128318BA2B9B
:103760008030A100C3308A0142201E30A60066309E
:103770008A017721023003178D000301831603139A
:10378000BC1A013083128A01672104308316480273
:103790008A150A168312031D082C8030A100803080
:1037A0008A0142201E30A60070308A0177218A15D6
:1037B0000A1683168310BC1D831483128318EA2B08
:1037C0008030A100C3308A0142201E30A600803024
:1037D0008A0177218A150A1683168310BC1983146F
:1037E00083128318FD2B8030A100C3308A01422050
:1037F0001E30A6008A308A017721033003178D001E
:10380000030183160313BC19013083128A01672157
:103810000530831648028A150A168312031D352CBB
:103820008030A10080308A0142201E30A6009430F2
:103830008A0177218030A100C5308A0142202B30D7
:103840008A010B2183164C0883128A0149201E30FD
:10385000A600A4308A017721043003178D00831657
:1038600003134C0883128A0167210630831648022D
:103870008A150A168312031D512C8030A100823054
:103880008A0142201E30A600AB308A0177218030A9
:10389000A100C1308A0142201E30A600B8308A0142
:1038A00077218A150A16D32A83163308CF0003011D
:1038B0008312871A0130CA000130071A03014A0532
:1038C0008A150A1603197B2C01308316B300871062
:1038D0008312871483160711831207118316871129
:1038E0008312871183160710831207100130831685
:1038F000CD000A30CE0083120130871A0301CA00BE
:103900000301071A01304A058A150A1603199F2C6C
:1039100002308316B30087108312871083160711B5
:1039200083120715831687118312871183160710D8
:10393000831207100B308316CD000C30CE0083129B
:103940000301871A0130CA000301071A01304A0532
:103950008A150A160319C32C03308316B300871087
:10396000831287108316071183120711831687119C
:103970008312871583160710831207100D308316E4
:10398000CD000E30CE0083120130871A0301CA0029
:103990000130071A03014A058A150A160319E62C95
:1039A0008316B301871083128710831607118312C1
:1039B000071183168711831287118316071083124C
:1039C000071401308316CD000C30CE00831283160D
:1039D0004F0833028A150A16831203191E2D831607
:1039E0004D08C2004D08C3004E08C40083128A115E
:1039F0000A1611278316B3088A150A168312031DA7
:103A00001E2D8A0138208030A10080308A0142209A
:103A10001E30A600C6308A0177218030A100C03058
:103A20008A0142201E30A600D6308A0177210B3051
:103A3000B500B8308A01B0218A013820080063003F
:103A40008A150A161F2D53005700520026005000F9
:103A50006F0077006500720020004D006500740063
:103A6000650072000000760031002E003100200059
:103A700062007900200050004100310052005500E2
:103A80004D000000200020002000320030003000F7
:103A900039002000560052005A004100000020006A
:103AA00052006100640069006F006B0061006D00EE
:103AB00070007700650065006B0000005300650032
:103AC0006C0066007400650073007400000057000D
:103AD00020002000200020002000200020002000E6
:103AE00000002000640042006D0020002000000063
:103AF0003E0031003A0035002E003000000020006A
:103B0000640042006D0020002000000020006400DE
:103B100042006D00200020000000430068006100AA
:103B20006E0067006500200053006500740074009B
:103B300069006E00670073003F000000200059001C
:103B40004500530020002F0020006E006F00000091
:103B5000200079006500730020002F0020004E0037
:103B60004F00000043006F00720072002E00200022
:103B70005B00640042005D00000057002000200050
:103B80002000200020002000200020000000200055
:103B9000640042006D002000200000004400490045
:103BA0005200450043005400000020002000200087
:103BB000430061006C0069006200720061007400E3
:103BC000650000003000640042006D00200020000D
:103BD000000044004900520045004300540000002A
:103BE00044006100740061003A00200000004400BD
:103BF0006100740061003A00200000004400610090
:103C000074006100200069007300200073007400DC
:103C10006F00720065006400210000005300650021
:103C2000740020005500700064006100740065009D
:103C30002000440065006C00610079000000300045
:103C4000300020006D005300650063002E0020004E
:103C500000004400650062007500670067006900AD
:103C60006E00670020006F006E003F000000200023
:103C700059004500530020002F0020006E006F0007
:103C80000000200079006500730020002F00200054
:103C90004E004F0000005000680061007300650096
:103CA000200043006F007200720065006300740022
:103CB00069006F006E00000020004F004E002000E1
:103CC0002F0020006F0066006600000020006F00DB
:103CD0006E0020002F0020004F004600460000002C
:103CE0002000560052005A004100200062006F0080
:103CF0006F007400200069006E0066006F00000015
:103D000020004F004E0020002F0020006F006600B2
:103D10006600000020006F006E0020002F002000D1
:103D20004F00460046000000430061006C0069003F
:103D30006200720061007400650020006C00650084
:103D4000760065006C0000002000640042006D00F9
:103D50002000200000005000750073006800200063
:103D600074006F0020006500780069007400000096
:103D7000730065007400740069006E0067007300D2
:103D800020006D0065006E007500000020004D00F1
:103D9000610078002E00200069006E007000750040
:103DA0007400200069007300200000002000200043
:103DB0003100570020002F00200033003000200089
:083DC000640042006D000000E8
:02400E00321F5F
:10420000050001000100010028000000000000007E
:1042100000000000000000000000010084005400C5
:10422000CC00CD008400690099009A0084006900E8
:1042300099009A00020084005600CC00CD00840052
:104240005400CC00CD008400690099009A0003005E
:104250008400580000000000840053003300330045
:104260008400690099009A0004008400580000004E
:10427000000084005400CC00CD0084006900990047
:104280009A000500840058000000000084005400DB
:10429000CC00CD008400690099009A0006008400DB
:1042A00058000000000084005400CC00CD008400C1
:1042B000690099009A00070084005800000000007F
:1042C00084005400CC00CD008400690099009A005D
:1042D0000800840058000000000084005400CC0056
:1042E000CD008400690099009A00090084005800FC
:1042F0000000000084005400CC00CD008400690060
:1043000099009A000A008400580000000000840010
:104310005400CC00CD008400690099009A000B0085
:1043200084007000CC00CD0084006F0033003300A7
:104330008400690099009A000C0084005200660015
:10434000660084004C00CC00CD0084006900990018
:104350009A000D00840052006600660084004C0044
:10436000CC00CD008400690099009A000E00840002
:1043700052006600660084004C00CC00CD00840032
:06438000690099009A009B
:00000001FF
